:020000040000FA
:100000006400A72085018514860188209B2000308C
:100010003A21A2205920B0200B1D11280E303A2180
:100020000628930130089200AC0031089100AD0021
:10003000C620061F062885105920B0203008AE00C3
:100040003108AF00851406165920A220861A3928D7
:10005000AD21861F322843305921DC20C42198214C
:10006000DE2037284C305921DC209D210F214421EE
:100070003F2893012C0892002D089100C620061FEE
:1000800003289B20B0203008031948280B1D4B285B
:100090000E303A212428AD21AB21861F542831305F
:1000A0003A219821DE20242836303A219C210F2144
:1000B00024285B205B200530A8006120A80B5D2868
:1000C00000347D30A900CB30AA00AA0F6528A90F03
:1000D000652800341830A600B201B301B401B5019F
:1000E000323084000430A700333080078019F039A3
:1000F000801B0F398002840AA70B7428910D920D82
:10010000930DB50DB40DB30DB20DA60B70280800FC
:100110005B208511051103305E215B2003305E21D9
:1001200003305E2102305E210C30A3200630A32074
:10013000992001309C280230A520F230A900FB3024
:10014000AA006528C030A520652985115A29831683
:100150003730810010308500E030860083120800BF
:10016000B001B1010B118101831605145B2005104C
:1001700083120108B00083160116000001128312D9
:10018000B103010830060319BB2808006A20463075
:100190005921DC20B2080319CF2848214A2133080D
:1001A000F0390319D4284C214E21502152214621E7
:1001B000542156212C303A293B303A2932080F3944
:1001C0000319E82857214C214E2146215021FB28B4
:1001D000330E0F390319F22857214E2146215021A1
:1001E0005221FB2833080F390319FD2857214621D6
:1001F0005021522154211C303A29340E0F39031D4D
:100200000829442134080F39031D092944210A29EA
:100210005021522154214621562120303A293208BA
:100220000F390319192957214C2146214E215021FC
:100230002229330E0F3903192429572146214E2133
:100240005021522124303A2933080F3903192E291D
:10025000572150215221462154213929340E0F397A
:10026000031D34294421352950215221462154218E
:1002700056212830890083160814831208080319B0
:1002800008005921890A3B29203059292E30592943
:10029000320E572932085729330E57293308572968
:1002A000340E572934085729350E572935080F3988
:1002B000303E8515AB002B0E5E212B080F39061A38
:1002C00010388600051500000511B330A900A90BF0
:1002D0006729A90B692900345D237129E522712959
:1002E00095222108990022089A0024089B00080002
:1002F0001908A1001A08A2001B08A40012089900FE
:1003000013089A0014089B000800120889001908B5
:10031000920009089900130889001A089300090837
:100320009A00140889001B08940009089B00080023
:100330006E21BC217021A4297021B5217021CA2110
:100340007821702185216E212D30931F2030592175
:10035000931339226A28CE21AE29CC21CA216E21DD
:1003600078217021C42185216C297821AB3094003B
:10037000383093004D30C22978218C3094001C30E5
:10038000930040309200080078219401930192017B
:100390000130D7292C30CF292E30CF29303084009E
:1003A00078219401930100089200840A00089100CA
:1003B000F8299F011308031DE3291208930003196C
:1003C000F32992019F151F089402031D031C512B52
:1003D0000310931BF029920D930D940BE929512BD7
:1003E000951F9313003493019201910194010034FD
:1003F000963094009501931F062A9109920993095A
:10040000910A0319920A0319930A95179F01130879
:10041000031D1B2A120893001108920091019F15D9
:100420001308031D1B2A1208930092019F111F1627
:1004300013080319F3291F089402031D031C512BF1
:100440000310931B292A910D920D930D940B212AD1
:10045000512B161B121CF029911FF029920A031927
:10046000930A031DF029930C920C940A0319DB2ABA
:10047000F02991011408031900341308950093170B
:1004800096309402941F892A9409940A0830140221
:10049000031C652A9400910D120891001308920024
:1004A000930108301402031C652A9400910D120870
:1004B0009100920108301402031C652A9400910DEA
:1004C00091011408031D03106E2A140803196E2AE3
:1004D0000310930C920C910C940B682A161B111CA0
:1004E0007A2A031C7A2A910A0319920A0319930A99
:1004F000931B892A951F0034930992099109910A47
:100500000319920A0319930A00349301920191018D
:1005100000341614961FFF349301951FFF3093008B
:1005200092009100950D930CFF341408031D1B08D5
:100530000319F32913081A0695001B0894077E3047
:10054000031CA62A94020318DB2AA92A9402031C7E
:10055000512B130891001208900091179A1703105D
:100560009301920110309F00101CBC2A19089207B9
:100570001A0803181A0F9307930C920C910C900C05
:1005800003109F0BB42A931BC92A910D920D930D52
:100590009403161B121CD82A911FD82A920A0319F9
:1005A000930A031DD82A930C920C940A0319DB2A90
:1005B000951F931300349614961FFF34FF30940058
:1005C00093009200950D930CFF341B0803195B2BCD
:1005D00014080319F32913081A06950093179A179C
:1005E0009F011308910012089000190890021A0840
:1005F000031C1A0F910291019001031C052B03109B
:10060000930C920C910C01309F001B089402031C68
:100610000F2B7E301F0794070318DB2A142B7E3024
:100620001F079407031C512B10309E00900D910D55
:10063000920D930D9F0D190892021A08031C1A0FB0
:1006400093021A0D9F041F1C272B10142E2B190820
:1006500092071A0803181A0A930710109E0B162BFC
:10066000161B101C4A2B0310920D930D9F0D190899
:1006700092021A08031C1A0F93021A0D1F04013963
:1006800090070318910A031D4A2B910C900C940AB1
:100690000319DB2A951F911311089300100892008B
:1006A00000341615961FFF34013094009301920117
:1006B000950D930CFF349615FF3480309A0613087D
:1006C0001A069F009101980114081B02031C7A2B43
:1006D0001B088F0014089B000F0894001A088F0055
:1006E00013089A000F08930019088F001208990048
:1006F0000F0892001B080319003413089500931784
:100700009A171B0814029B000319A02B08301B0228
:10071000031C972B9B00190898001A0899009A014E
:1007200008301B02031C972B1508930000341B088C
:100730000319A02B03109A0C990C980C9B0B9A2B65
:100740009F1FAA2B980999099A09980A0319990ACF
:1007500003199A0A1808910719080318190F920724
:100760001A0803181A0F93079F1BBE2B031C292A74
:10077000930C920C910C940F292ADB2A0318062A59
:10078000910992099309910A0319920A0319930A8C
:0607900080309506D92916
:02400E00F23F7F
:1042000020002000630061006C0069006200720001
:104210006100740069006E0067000000200020004B
:1042200020004F00760065007200200052006100FF
:104230006E0067006500000020006E004600000070
:10424000200070004600000020006D0048000000C3
:10425000200075004800000020004B0048007A0054
:104260000000430020003D00200000004C00200022
:104270003D00200000007200650066002000000084
:00000001FF
